:100000005FC177C176C175C174C173C172C171C15D
:1000100070C16FC16EC16DC16CC16BC120204475D0
:10002000616C2D53656E736F722020202052462024
:10003000506F7765726D6574657220204453504D22
:10004000303320205665727320312E3428632920E6
:10005000323030342020444C354E4547002020417A
:1000600044432D72617776616C75652020666F72EE
:100070002063616C6962726174696F6E2041443003
:10008000204144312041443220414434202D2D2D43
:10009000202D2D2D202D2D2D202D2D2D200044699E
:1000A0006F64652D53656E736F722020202061622E
:1000B000733A203A78782E78782064426D20726501
:1000C0006C3A203A78782E78782064422020207884
:1000D000787878202073656E736F72202D2000541D
:1000E0006865726D616C2D53656E732E782020618A
:1000F00062733A203A78782E78782064426D2072C4
:10010000656C3A203A78782E787820644220202056
:1001100020202020202020202020202020202000FF
:100120004261747465727920566F6C7461676520E2
:10013000202020202D2E2D20566F6C74732020201F
:1001400020205374617475733A202D6F6F2D202019
:10015000202020202020202020202020202020209F
:10016000005741524E494E47204F5645524C4F4141
:1001700044202072656475636520696E7075742013
:100180002020706F77657220746F2061766F6964CC
:100190002064616D616765206F662073656E736FA3
:1001A00072005072652D417474656E756174696F6B
:1001B0006E207365743A203A78782E7878206442FD
:1001C00020207573652052656C2D5265736574200F
:1001D0002620205A65726F2D41646A20746F207347
:1001E0006574000400060007000A000C00100013EC
:1001F0000018001D0023002A0033003C0047005374
:10020000006200720085009B00B300D000F0001473
:10021000013E016D01A201E00124027F022C03FFD7
:10022000FF0300040005000600070009000B000E94
:1002300000120016001C0023002C0037004400555B
:1002400000690081009E00C200EC001E015A019F5F
:1002500001F1015002C0024103D703FFFF15001650
:100260000018001A001C001F00230028002E003672
:100270000040004C005C006F008800A600CC00FB32
:100280000036017F01D8014502C9026703FFFF164E
:1002900000170019001B001E00220027002D00344B
:1002A000003D00490058006A0082009F00C400F32E
:1002B000002E017801D5014A02DE029703FFFF00FC
:1002C00011241FBECFEDCDBF10E0A0E6B0E0EEE3FD
:1002D000FFE003C0C89531960D92A436B107D1F75F
:1002E00010E0A4E6B0E001C01D92A23BB107E1F727
:1002F00001C086CECFEDD0E0DEBFCDBF1FEF11BB7A
:1003000080E284BB86E087BB89E388BB83E88FBD3E
:1003100001E00EBD80E092E090936D0080936C0050
:1003200082E08BBD80916C008ABD5ED5802FC4D2E7
:100330007BD5812F9AD2812F98D2812F96D283E0BC
:1003400080936000B9D270D580916700882371F1E5
:100350008091640064D2082F192F8091670081304A
:1003600029F40031110510F01092670080916700A8
:100370008F3F29F40131110510F41092670080912C
:100380006700282F332727FD309580916C009091CE
:100390006D00820F931F90936D0080936C00892FE6
:1003A000990F990B8BBD80916C008ABD86B3082F85
:1003B000112703FF0FC005FF0DC010926800809148
:1003C000690090916A00009729F0019790936A0064
:1003D0008093690000FD0BC0809160008F5F809367
:1003E0006000873018F082E080936000E4D204FD62
:1003F00025C0909160009330A1F48091620081301B
:1004000019F41092620005C080916100813021F4DE
:100410008F5F8093610005C081E0809361008093CD
:100420006200953051F480916400882319F0109295
:10043000640003C084E080936400BDD203FD52C019
:1004400080916000843009F044C0809165009091F3
:10045000660027E1803792070CF044C0282F392F1F
:100460002F5F3F4F309366002093650090916800A6
:10047000892F8F5F809368008A3040F090936800E6
:1004800082E390E090936A00809369008091690014
:1004900090916A00892BD1F0932F822F64E670E04F
:1004A00025D5892B69F02F5F3F4F932F822F64E66C
:1004B00070E01CD5892BB9F7309366002093650056
:1004C00082E390E090936A00809369008EE1CDD141
:1004D00009C080916E0090916F009093710080939D
:1004E000700069D205FD61C080916000823011F01A
:1004F0008530A1F480916700882381F480916400A5
:100500008ED1082F192F419718F08FEF8093670035
:100510000031110518F481E080936700809160003C
:10052000843009F042C0809165009091660028EE09
:1005300081399207D4F1282F392F21503040309340
:1005400066002093650090916800892F8F5F8093EB
:1005500068008A3040F09093680082E390E09093C6
:100560006A00809369008091690090916A00892BEC
:10057000D1F0932F822F64E670E0B8D4892B69F014
:1005800021503040932F822F64E670E0AFD4892B46
:10059000B9F7309366002093650082E390E0909372
:1005A0006A00809369008EE160D180916000992794
:1005B0008430910509F4A2C0853091053CF4823065
:1005C000910561F0039709F47BC0BDCE853091059C
:1005D00009F498C0069709F4EFC0B5CEA1D380E026
:1005E0001ED1082F192F8F705BD18093A400E4E0F7
:1005F00016950795EA95E1F7802F8F7051D180937A
:10060000A30074E0169507957A95E1F7802F8F7017
:1006100047D18093A20081E002D1082F192F8F705B
:100620003FD18093A80064E0169507956A95E1F79D
:10063000802F8F7035D18093A70054E016950795D1
:100640005A95E1F7802F8F702BD18093A60082E01E
:10065000E6D0082F192F8F7023D18093AC0044E08F
:10066000169507954A95E1F7802F8F7019D18093E1
:10067000AB0034E0169507953A95E1F7802F8F701F
:100680000FD18093AA0084E0CAD0082F192F8F7051
:1006900007D18093B00024E0169507952A95E1F7DD
:1006A000802F8F70FDD08093AF0094E01695079552
:1006B0009A95E1F7802F8F70F3D08093AE0043CEF0
:1006C00080916100ACD0082F192F8091620088239F
:1006D00089F00332110518F482E080936100085D0F
:1006E000134018F081E0809361008091610097D001
:1006F000082F192F912F802F33D225CE80E090E044
:1007000061D121CE809164008AD0082F192F28D280
:1007100080916B00813009F416CE0031110539F457
:100720008CE38093A9008EE38093AA000CCE013164
:10073000110508F1312F202F295D3F4F203431055D
:1007400014F02FE330E0F32FE22FEE58FF4F8EE34B
:10075000808347E3283331050CF4F5CDE42FFF27E0
:10076000EE58FF4F8DE280834F5F842F99278217C9
:100770009307A4F3E8CD312F202F285D3F4F20337E
:10078000310514F420E330E0F32FE22FEE58FF4F51
:100790008CE3808348E3283331050CF0D4CDE42F7B
:1007A000FF27EE58FF4F8DE280834150842F992719
:1007B00028173907A4F3C7CD83E031D0082F192FAC
:1007C0008158924028F084E680939F0087E604C019
:1007D00082E780939F0080E780939C0083E01695DA
:1007E00007958A95E1F780E090E020E00A962F5F78
:1007F00008171907D8F72150081B190BE02FE65FDF
:100800002A3018F02A5081E301C080E280938500ED
:10081000205D20938600E05DE093880094CD1F93D7
:10082000CF93DF93982F86EE86B997B9C0E0D0E0DA
:1008300010E00CC081E019D024B185B19927982F20
:100840008827820F911DC80FD91F1F5F84E0B4D283
:10085000181780F3A4E0D695C795AA95E1F78C2FD9
:100860009D2FDF91CF911F9108951F93CF93182F44
:1008700012BE83E083BFC0E0C11778F481E09CD250
:10088000982F88B7892339F0CF5F81E095D2982FD0
:1008900088B7892B88BFC11788F3CF911F9108951E
:1008A000805D8A3308F0895F99270895843209F4BE
:1008B00082E0805899270895AF92BF92CF92DF923D
:1008C000EF92FF920F931F93CF93DF93C82EDD24F7
:1008D00012E7A12E10E0B12EC1E6EC2EC1E0FC2EF5
:1008E00000E211E0CFEDD0E0A2EAB1E06EE970E005
:1008F0004DE550E02CE130E08C2D992784309105B6
:1009000021F1853091054CF482309105A1F08330BE
:100910009105B4F4019751F02EC086309105F9F09D
:1009200086309105BCF00797F9F025C0F32FE22F30
:10093000C895802D1DC0F52FE42FC895802D18C0B7
:10094000F72FE62FC895802D13C0FB2FEA2FC895EF
:10095000802D0EC0FD2FEC2FC895802D09C0F12FE2
:10096000E02FC895802D04C0FF2DEE2DC895802D59
:10097000FB2DEA2D8083D3942F5F3F4F4F5F5F4F56
:100980006F5F7F4F119621960F5F1F4F0894E11CF8
:10099000F11C0894A11CB11CFFE3FD1508F0ACCFBD
:1009A000DF91CF911F910F91FF90EF90DF90CF904B
:1009B000BF90AF900895809160007EDF35D289E1CD
:1009C00054DF08952F923F924F925F926F927F92E1
:1009D0008F929F92AF92BF92CF92DF92EF92FF924F
:1009E0000F931F93CF930091650010916600800FC5
:1009F000911F90936F0080936E00C0E02090600084
:100A0000A0907000B09071003090870040908800F6
:100A100050908900F0918B00A0918C00C0906900EB
:100A2000D0906A0060909700709098008090990034
:100A300090909B00E0909C00282F392FF22C44E0EE
:100A4000241619F4312F202F04C0CC2311F02A19B9
:100A50003B0937FF05C0309521953F4FBDE201C0EE
:100A6000BBE240E050E0E0E02417350734F04851A5
:100A70005C4FEF5F24173507D4F7E150241B350B8B
:100A800028513C4F40E050E070E02417350734F027
:100A90004C595F4F7F5F24173507D4F77150241BE3
:100AA000350B2C593F4F40E050E060E024173507EC
:100AB00034F0465F5F4F6F5F24173507D4F76150FE
:100AC000241B350B265FCC2319F034E0F31689F490
:100AD0003B2E40E3442E4E0E30E3532E570EF62F9E
:100AE000F05DA22FA05DC114D10481F0FFE5AF2F0E
:100AF0000DC06B2EB0E37B2E7E0E50E3852E870E4D
:100B000040E3942E960E30E3E32EE20ECF5FC23028
:100B100008F492CFE0929C0090929B008092990002
:100B20007092980060929700A0938C00F0938B00D5
:100B3000509289004092880030928700CF911F9197
:100B40000F91FF90EF90DF90CF90BF90AF909F906C
:100B50008F907F906F905F904F903F902F9008956F
:100B6000BF92CF92DF92EF92FF920F931F93CF939A
:100B7000DF93E82EF92EBB24C0E0D0E00C2F1D2F10
:100B8000CC2EDD2E8091600097DECAD0B0926B0033
:100B900080916000833009F03FC080916100813016
:100BA000E9F401C0B394CB2DDD27CC0FDD1F0C2F52
:100BB0001D2F0D511E4F912F802F08D1E816F906D9
:100BC00088F7E2EFCE2EEFEFDE2E912F802FFED0B2
:100BD000082F192FCF51DE4F1AC0B394CB2DDD272C
:100BE000CC0FDD1F0C2F1D2F0F5D1D4F912F802F60
:100BF000EDD0E816F90688F772EEC72E7FEFD72EF4
:100C0000912F802FE3D0082F192FC15EDD4F8C2F3D
:100C10009D2FDCD0D92FC82F80916000853009F03E
:100C200042C0809164008823E9F4B82E01C0B394D7
:100C3000CB2DDD27CC0FDD1F0C2F1D2F035A1D4F91
:100C4000912F802FC3D0E816F90688F76DEFC62ED6
:100C50006FEFD62E912F802FB9D0082F192FC55A9C
:100C6000DD4F1CC0BB2401C0B394CB2DDD27CC0FBE
:100C7000DD1F0C2F1D2F01571D4F912F802FA6D048
:100C8000E816F90688F756EFC52E5FEFD52E912F9F
:100C9000802F9CD0082F192FC357DD4F8C2F9D2FED
:100CA00095D0D92FC82FBB2059F48CE380938600B0
:100CB000809396009D2D8C2D64E670E005D125C0B3
:100CC0008FEF0F3F180731F487E0F6DD81E0809366
:100CD0006B001CC00C1B1D0BEC1AFD0A9F2D8E2DEA
:100CE00064E670E0F1D0712F602F00D1262F372FEE
:100CF000CB0CD11C9D2D8C2D64E670E0E5D0280F27
:100D0000391F24563040932F822F5CDEDF91CF9124
:100D10001F910F91FF90EF90DF90CF90BF900895BB
:100D200020916000233001F580916200882359F002
:100D300081E68093A30085E78093A40084E78093F5
:100D4000A5008FE60AC08DE68093A30081E680931C
:100D5000A4008EE68093A50080E28093A600809197
:100D60006100805D8093B000253049F4809164007B
:100D7000882311F481E301C082E380937F0080E245
:100D800080938100233011F0253049F48091650073
:100D900090916600892B19F081E4809381002230C4
:100DA00011F0253039F480916700882319F08AE525
:100DB0008093810008950895282F81E090E002C07B
:100DC000880F991F2A95E2F799270895F92FE82FA0
:100DD0003196C895802D31979927982F8827C895E7
:100DE000202D820F911D0895CF938AE03EDD85B3BB
:100DF0008F7C85BBC1E080E35AD081E036DDCF5FD8
:100E0000C430C8F388E353D081E02FDD8CE04FD0AD
:100E100081E02BDD81E04BD084E027DD82E047D00C
:100E200084E023DDCF9108950F931F93CF93AD9866
:100E300080E83DD084E019DDAD9AC0E002E710E023
:100E4000F12FE02F81910E2F1F2F31D0CF5FC031B6
:100E5000B8F3C0E202E910E0F12FE02F81910E2FEC
:100E60001F2F25D0CF5FC033B8F3AD9880EC1FD0D3
:100E700084E0FBDCAD9AC0E102E810E0F12FE02F46
:100E800081910E2F1F2F13D0CF5FC032B8F3C0E374
:100E900002EA10E0F12FE02F81910E2F1F2F07D0D3
:100EA000CF5FC034B8F3CF911F910F91089582BBEB
:100EB000C29AC29882E390E001D00895009711F0A1
:100EC0000197F1F7089508955527002480FF02C087
:100ED000060E571F660F771F6115710521F0969555
:100EE0008795009799F7952F802D089597FB092EE8
:100EF00007260AD077FD04D00CD006D000201AF4C3
:100F0000709561957F4F0895F6F7909581959F4F65
:100F10000895AA1BBB1B51E107C0AA1FBB1FA61740
:100F2000B70710F0A61BB70B881F991F5A95A9F792
:0E0F300080959095682F792F8A2F9B2F08951A
:040F3E0001010100AC
:00000001FF
